:020000040000FA
:04000000B3018C2993
:080008009229A50038088400CC
:100010003608F820841300052D1C36060319232802
:100020002508031D1B282B08FF3E031C24280A302B
:100030000C212B082428250AFF3003192328250B1F
:1000400023282C082428AE09AE0C8729B316B31E2A
:10005000B312B3192F28B315682003185628083097
:10006000A4007C20A30DA40B3128B31E61208620A0
:100070008220B31A56205B20230803108729B31669
:10008000B31EB31233194928FE39B40033150310D7
:100090008729331A5128A7003316682003185628D9
:1000A00027086F2003185628B31E87296120862051
:1000B00033113312B31138088400360884178004D2
:1000C00067283808840036098005841780050800F1
:1000D0005B208620612082203408B3190138A300F8
:1000E0000830A400A30D03185B20031C61208620A8
:1000F0008220A40B72285B208620380884003608F2
:100100000005FF3E39088400370964283908840057
:1001100037085E28A601A500B4172730A4001030C8
:100120009D200330A400E8309D20A40164309D2070
:10013000A4010A309D202508A828A3002608A200B3
:100140002508A10055212108031DB413B41B080084
:10015000303EA80085130513051383168513051378
:100160000513F030850583122808B318D4283A30D7
:10017000A200FC301A213330A700E9201030A20081
:1001800068301A21E920643019212230A700E920C3
:100190002830D3200C30D3200130D3200630D32098
:1001A000B3142808D4283314A700331CE2280513FD
:1001B000033C031CE728E7200530A200DC301A21AD
:1001C000031408003314FE3C031987290517A70EF2
:1001D000331C33108517F030850527080F39850447
:1001E0008513A70E3318E9282C30192103140800B1
:1001F00084178004872983169B001C141A088729FA
:1002000083169A001C1555309D00AA309D009C1441
:100210009C1808291C118729A401A300FF30A307FB
:10022000031CA407031C87290330A200DF301A2116
:100230000E29A201E83EA100A209FC30031C2329DB
:10024000A10703182029A1076400A20F2029211863
:100250002929A11C2D2900002D290800A300033005
:100260003729A30001303729A30004303729A9001A
:1002700024082202031D3E2923082102043003180A
:100280000130031902302905031DFF308729A3001F
:100290002108A7002508A1002708A5002208A7001B
:1002A0002608A2002708A6005729A601A50110309C
:1002B000A700220DA50DA60D2308A5022408031CE6
:1002C000240FA60203186B292308A5072408031886
:1002D000240FA6070310A10DA20DA70B5929210871
:1002E00087291030A900A201A101A80CA70C031CAA
:1002F0007F292308A10724080318240FA207A20CB2
:10030000A10CA60CA50CA90B752925088729831318
:1003100003138312640008008316061786178616D7
:100320008312052AA000030E8301BA000A08B50053
:10033000861B4F16861F4F12861BCF16861FCF12A5
:10034000861B4F17861F4F13861BCF17861FCF1391
:10035000061B4F14061F4F10061BCF14061FCF108D
:10036000061B4F15061F4F11061BCF15061FCF1179
:1003700064004F0851020319FD2964004F08003C36
:10038000031DD52964005008F03C031DCB29CC0186
:100390000130CE00D329640050080F3C031DD3293F
:1003A0000130CC00CE01D101FD2964004F080F3C83
:1003B000031DDD290F30D000FD2964004F08F03CFB
:1003C000031DE529F030D000FD2964004F08FF3CF3
:1003D000031DFD29640050080F3C031DF329CC01C7
:1003E0000130CE00FB2964005008F03C031DFB29BE
:1003F0000130CC00CE01FF30D10035088A003A0E22
:100400008300A00E200E0B10090007309F008316FA
:1004100081018312C230C900C330CA000130A40078
:10042000F4300D21FE30A9200130A9205030A92040
:100430004C30A9204C30A9202030A9205630A920CA
:100440003330A9206130A920FE30A920C030A92076
:100450004430A9204C30A9203130A9204D30A920AA
:100460004630A9204B30A9202030A920CC01CE0154
:100470000130A400F4300D210030FB20C500013014
:10048000FB20C6000230FB20D3000330FB20D2004B
:100490000630B8000230B6000630B9001030B700A0
:1004A000490841204608412045084120C2303F20EC
:1004B00088308B000630B8000230B6000630B90034
:1004C0001030B70049084120460841204508412026
:1004D000CE303F20D023082464004E08013C03198D
:1004E0009E2A64004C08013C0319B22A0630B80069
:1004F0002030B600AD01FF30AB00AC010130AE00E2
:100500004B080520CB000318C52A0630B80002307E
:10051000B6000630B9001030B7004A084120262046
:10052000CD00FE30A9208730A92064004D1F9B2AF2
:100530004C30A9209D2A5830A9206C2ACE0152089F
:10054000C5070318C60A4508A1004608A2007D3069
:10055000A40000303421031DB12AA030C5000F30A3
:10056000C600572CCC015208C502031CC60345081F
:10057000A1004608A2000F30A400A0303121031DC5
:10058000C42AC5017D30C600572CFE30A920013099
:10059000A920FE30A9208030A9205E30A92020307B
:1005A000A9205330A9207430A9206530A9207030CB
:1005B000A920FE30A920C030A9207630A920203003
:1005C000A9207830A9202D30A9204D30A9206130F4
:1005D000A9206C30A92064004E08013C031DF22ABA
:1005E000CE016A2B64004C08013C031DF92ACC01A2
:1005F000092B0630B8002030B600AD01FF30AB004B
:10060000AC010130AE004B080520CB0003185A2A7C
:10061000EB2AFE30A9200130A920FE30A92080302D
:10062000A9204630A9206130A9206B30A920743060
:10063000A9206F30A9207230A9203A30A920640087
:100640000A3053020318262B2030A920FE30A9209F
:10065000C030A92053088A202D30A9206630A92057
:100660006130A9206330A9206830A92064004E08B9
:10067000013C0319502B64004C08013C03195A2B10
:100680000630B8002030B600AD01FF30AB00AC0141
:100690000130AE004B080520CB000318C52A362BCD
:1006A000CE01D30A64000B305302031C592B0130D6
:1006B000D300632BCC01D303640001305302031831
:1006C000632B0A30D300831602309B008312530839
:1006D0000021092BFE30A9200130A920FE30A920DD
:1006E0008030A9205330A9207430A9206530A9207A
:1006F0007030A9203A30A920FE30A920C030A920AE
:100700007D30A700A8015208A300A4017121C700F1
:100710002608C8004808A60047088B206B30A9208F
:100720004830A9207A30A92064004E08013C031902
:10073000AE2B64004C08013C0319BF2B0630B800F7
:100740002030B600AD01FF30AB00AC010130AE008F
:100750004B080520CB000318C52A942BCE01520864
:10076000A700A8010230A300A4017121D2006400F7
:1007700041305202031CBE2B0130D200C92BCC01E8
:100780000310D20C6400013052020318C92B403010
:10079000D200831603309B008312520800216A2B7B
:1007A0007D30A700A8015308A300A4017121BD005A
:1007B0002608BE004508A7004608A8003D08A3007B
:1007C0003E08A4007121BB002608BC000330A40031
:1007D000E8304721C1002208C2004508A7004608AA
:1007E000A8005308A300A4017121C3002608C40077
:1007F0000730C3050030C4054308A7004408A8001B
:100800007D30A300A4017121BF002608C0000800AC
:10081000FE30A9200130A920FE30A9208030A92077
:100820004108A1004208A2002730A40010302E2168
:10083000031D282C2030A9204108A1004208A20055
:100840000330A400E8302E21031D282C2030A920DD
:100850004208A60041088B202E30A920FE30A92096
:10086000C030A9203F08A1004008A200A4016430C4
:100870002E21031D482C3030A9203F08A10040083C
:10088000A200A4010A302E21031D482C3030A920DB
:100890004008A6003F088B202030A9204D30A92019
:1008A0004830A9207A30A9202030A92008008316DA
:1008B0009B01831245080021831601309B0083129F
:0608C000460800215A2A3F
:02400E00703F01
:0842000000002800010001008C
:00000001FF
